:1074000080E189BD82E189BD09B400FEFDCF089508
:10741000AA2069F08091E9008F931092E9009FD42F
:1074200083FF01C01ED58F9187708093E900089576
:107430008EEF0090E10008220092E1000895F20131
:10744000F999FECFF2BDE1BD0895F9DFF89A80B554
:1074500008C0F5DF1FBA80BD0FB6F894FA9AF99A02
:107460000FBE31962F010895E0E0F0E085919491F0
:10747000019608958BEA34D0109289008AEF8093A8
:10748000880082E080936F0083E080938100E9E8C8
:10749000F7E785913AD0E539E1F781E08093D700AD
:1074A0008AE482BF1092D8001092E2001092DA00B3
:1074B0001092E10080E808D019BCAA241092E000E4
:1074C00064D489E055D481E98093D8000895A3E677
:1074D000B1E090E81AD08D939A95E1F7089586E08F
:1074E00008D010C083E005D08F2F0FD08E2F0DD085
:1074F00080E05E9A599809C005D085E0FADF05D092
:1075000080FDFDCF599A5E9808958EBD8DB587FF99
:10751000FDCF8EB508958FE08221E9F7F3DFE3E632
:10752000F6E090EB5C98892FF0DF80E1EEDF5C9A6B
:107530008191EBDF83E68E278F77D1F79395983B88
:1075400089F70895E3E6F1E097FC36C094FC4DC05E
:1075500092FE089596849920D1F3F894C089D78536
:1075600020E030E080E090E4AFEFBFEF11968919A2
:107570009040E0F72D01BD4F8D0127FD13C0E0E0E5
:10758000F8E011928EE7819392E4E11791939AE5E6
:1075900008F092E4E334C9F781931082BFDFFE0163
:1075A0002196A0DF94DFF901FED420583F4F040D4F
:1075B000151D9A9411F704C28301282D60906C0167
:1075C00070906B0143D019F48823C1F708953801F6
:1075D00088243CD0C9F580916A01821709F483019F
:1075E00060906E0170906D01F4CF80E1982E6090F4
:1075F0006E0170906D012AD059F48823B1F7089577
:107600009FEF95FC03C096FE089591E097FB890ECD
:10761000662477248301222719D0B1F48823A1F3AB
:1076200080916A0136F0881650F4821730F02130CC
:1076300003C0881520F4281710F48301282F6090C8
:107640006E0170906D01E8CF3801822EF3014ADFA0
:107650003EDFC3E6D1E0E2E8F7E70990859108163E
:1076600021F4E938D1F7088080104CCFC9E031DF30
:10767000CA95E9F7D0E197FC55C094FC37C096FE57
:107680001AC0C3E6D2E0E3E6F6E098E088E78E0FA2
:1076900000840192E817E1F7884F09900192E817FA
:1076A000E1F7C858DF4F9A9589F735DFC85FD340B7
:1076B000C33E49F749C0C3E6D6E0EBE5FAE098E0FF
:1076C0008E2F885702900086E817E1F738960A90C7
:1076D0000292E817E1F73897C857D0409A9581F79A
:1076E0001ADFC850DC4FC33E41F72EC0A3EEB6E010
:1076F000E3E6F6E09AE0C6E00D9080818025807F89
:10770000802582958193A336B90709F4B2E0E33668
:10771000F90709F4F2E0E336FC0771F7FCDEDA95CD
:1077200029F712C0A3EEB9E0E3E6FAE092E00E908A
:10773000829180258F70802582958083E336F907BA
:10774000B1F7E9DEDA9571F788270895E8EBF0E004
:1077500081818C7F81838CE0808374E0720D84EA68
:1077600002C0838384E88483848187FD0895721135
:10777000FBCF089502D084E9848388E08A95F1F7ED
:10778000089541524455424F59D5F08D14A1C881F6
:06779000CFD9F1AF0000AB
:10779600120110010200000841233600010000001A
:1077A600000109023E0002010080320904000001C6
:1077B6000202010005240010010424020405240627
:1077C6000001070582030800FF09040100020A0000
:1077D60000000705040210000107058302100001DE
:1078000011241FBE04B714BE88E18093600010925B
:1078100060008EEF9AE09EBF8DBF222433242101A9
:107820003101410180E887C00F928F939F931F928F
:107830000FB60F9211244F936F938091DA0080FF5F
:1078400034C020C00F920FB68F939F93EF93FF9396
:1078500088278093850080938400E0E5F1E09081A3
:107860008917980B908309F45D9A91818917980B79
:10787000918309F4289A239411F48315381EFF91FB
:10788000EF9154C08091D80080FF0FC08091DA0042
:107890008E7F8093DA008091D90080FF04C0B0DD34
:1078A00081E0A82E02C019BCAA248091E10080FFCB
:1078B0000BC058D280FF08C058D28091D800806297
:1078C00003DE19BC85E0A82E8091E10084FF1AC078
:1078D00049D284FF17C094DD8091D8008F7DF4DDFC
:1078E0008FEEA7DD3FD28F7E816042D2809153011F
:1078F000882331F48091E30087FD02C081E001C05C
:1079000084E0A82E8091E10083FF0CC02BD283FF7E
:1079100009C087EF8EDD82E0A82E1092530188DD2A
:1079200024D233D26F914F910F901F909F918F91DE
:107930000FBE0F9018958093610010926100B1E026
:10794000B5BF82E085BF81EF85B987EE84B91DB8E8
:10795000769A10BA83EF81BB83E68BB982EF8AB93E
:1079600080E58CBDBDBDA0E0E6E9F7E705900D928E
:10797000A035E1F71D92BB30E9F75F9A00FD7C9BD3
:1079800002C072DDE9F476DD789460DEB0D040DDCF
:107990008FB18095807F66991C9B8460982E30DE25
:1079A0008110D0DD92FC0AC08FE08221882921F469
:1079B0008091720187FF19D0332042F755DD31F3F2
:1079C000F89489EB8DDD81E08093E00010926F00E8
:1079D00010928100109285001092840081E085BF92
:1079E00015BE5D9A289A0C940000E5E0F0E07ADD7F
:1079F000A3E6B2E0C8E06DDDCA95E9F7A7DE80ED49
:107A0000B0DE80E0AEDEB6DEAADE81EDAADEC4E73F
:107A1000D1E0DE0184ECA7DE83818D93AA37D1F714
:107A2000A1DE83818D93A6DE1482AFE2B6E08D8164
:107A300017D08C8115D08E8113D09A8190748A8151
:107A400019F08F7184FF80560BD0898109D088810D
:107A500007D0992321F08A818695807102D05ECD6E
:107A600000D09E01DD91CD91CD59D94FFD91ED9181
:107A7000ED59FE4F41915191549F8295682F6F703F
:107A8000609DE00DF11DBE01152E8E0103561640BE
:107A9000143050F401900882C058DF4F1A94A9F7AF
:107AA000EB0121964A9579F7E901089556D107C06F
:107AB00009D102C0AA2039F052D182FFFBCF85FF45
:107AC000F7CF8091F1000895082E83E047D185FD1E
:107AD00007C03CD102C0AA2049F041D180FFFBCFB2
:107AE0000092F1005D9884E680935001089535D1AD
:107AF00082FFEAC0289884E680935101D7DF182FCF
:107B0000853431F422248EE7382E99DC8DE0C5C00F
:107B1000843511F4CBDFFACF8C34C1F38035B1F367
:107B2000843711F480E0B9C0813429F4BFDF582EC6
:107B3000BDDF482EEBCF833539F4E2E8F7E78591D6
:107B4000C3DFE938E1F7AAC0863521F482E3BCDF60
:107B500081E3A3C08A3649F48FE9CBDCC3E0D5DCEE
:107B6000B3DFCA95E1F7CEDC99C0833731F487E8FB
:107B7000ABDF85E9A9DF8EE190C0823631F489E57B
:107B8000A3DF80E0A1DF80E888C0823419F0873667
:107B900009F06FC033248ADFD82F88DFC82F86DF33
:107BA000082F8354843008F077C0063411F4440C55
:107BB000551CF20110926F001736B9F4033489F4A2
:107BC00083E091DCA2DC8EB51EBC7EDF0DB4219774
:107BD000D1F798DC08C0063411F4859101C035DC7A
:107BE00073DF2197C2F72F013CC00334A9F4E111E0
:107BF00004C075DC88ED77DC7FDC71DC82E073DC4F
:107C000055DF0DB48EBDCA95D9F731967FDC74DC93
:107C1000DA9569F72F0123C00634C1F49F01F437C8
:107C2000A8F4D4D113C042DF063461F4C0FB46F09F
:107C3000F43728F4182E81E087BFE8951124329696
:107C4000082E04C0043409F401C003DC21975AF75C
:107C5000063429F42F01F901F43708F4B5D18DE089
:107C600033DF063411F45694479482E080936F001A
:107C700015C08237E1E049F08634E0E031F08E341F
:107C8000E3E019F0813531F4E2E0F0E089E087BF0C
:107C9000849103C08B3111F08FE316DF83E0C5DBE5
:107CA00055D095FF03C009C0AA2071F058D080FFBD
:107CB000FBCF4CD002C0AA2039F051D080FFFBCFBF
:107CC00084E0B3DB8BE743C00895E4E5F1E067E0CF
:107CD00090915B0180915C01913231F0913AE1F534
:107CE0008132D1F55ED181C0823271F48191805BA5
:107CF0008191844089F580915D0180FD2DC0F894CB
:107D000081E08093E0007CCD803231F54AD1AA2019
:107D1000E9F08530D9F023D083FD18C082FFF7CF7A
:107D200004C0CFDE8193615031F09091F3008091D7
:107D3000F200892BB1F7C6DF611549F704C0AA200C
:107D400029F0853019F00BD080FFF9CF8EE79091A4
:107D5000E80089238093E800089584E066DB809141
:107D6000E80008958091E2000895FCDF8E7F806135
:107D70008093E200089582E061EC09D083E061E83D
:107D800002D084E060E842E103C080E060E042E0CD
:107D90004CDB81E007D01092ED006093EC00409343
:107DA000ED0008959091EB00892B8093EB000895EE
:107DB00060E0923029F0913029F4E0E062E102C005
:107DC000E2E16EE3F1E0089580915B0188234CF4D9
:107DD00002C0AA20C1F3C3DF82FFFBCF73CFAA206A
:107DE00091F3BDDF80FFFBCFB1CF40916101509196
:107DF00062014617510520F0462F611509F4A6DFF0
:107E000050E022C0AA2061F1853051F1A8DF83FD46
:107E100059CFA5DF82FD21C080FF16C03091F3004D
:107E20002091F20006C081918093F10041502F5FB4
:107E30003F4F411519F028303105A8F350E02830A4
:107E4000310509F451E082DF4115E1F65523D1F601
:107E500004C0AA2029F0853019F081DF82FFF9CF14
:107E600031CFEBE5F1E02DDE8193E336E1F72DDF55
:107E700076DF83FF91C080915B0190915C0191302E
:107E800009F170F09330F1F0953009F444C0963068
:107E900009F456C0983009F460C0993059F767C0AA
:107EA000823841F780915F01BFDA2091EB00109298
:107EB000E90077D02295269521702093F100109249
:107EC000F10052C0882311F08230A1F68F71823008
:107ED00089F680915D018823D1F420915F0127709C
:107EE00049F22093E9008091EB0080FF10C09330AD
:107EF00011F480E20BC080E155DF81E0880F2A9504
:107F0000E9F78093EA001092EA0088E04BDF1092D4
:107F1000E90047D02AC0882391F410915D011068D0
:107F20000FB7F8943ED050DF1ADF80FFFDCF1093DB
:107F3000E300103883E009F482E0A82E0FBF2CC0C4
:107F40008058823048F580915D0190915E0130DF6C
:107F5000603011F126D049DF1FC08038E9F421D00C
:107F6000809153018093F100F1DE2EDF15C088234C
:107F700099F490915D01923078F49093530111D06F
:107F800023DF80915301882321F48091E30091E065
:107F900087FD94E0A92EEFDEE2DE83FF089580E204
:107FA00001DF87EFD4CEA3E6B1E0F437B8F40ED00A
:107FB00090E40D901D9081E087BFE89532969A95E8
:107FC000C1F71124E058F04085E001C083E001D002
:0E7FD00081E187BFE89507B600FCFDCF08955C
:067FFA003231D6CFFBDCA2
:040000030000740085
:00000001FF
